:100000000EC028C027C026C025C024C023C022C0DF
:1000100021C020C01FC01EC01DC01CC01BC0112499
:100020001FBECFE5D2E0DEBFCDBF10E0A0E6B0E05E
:10003000EAE9FFE102C005900D92A838B107D9F7AF
:1000400011E0A8E8B0E001C01D92A432B107E1F7C9
:1000500050DAA2CFD5CF89E288BB089520917700EE
:10006000309178004091790050917A000CDF20E0C7
:1000700030E040E050E004C02F5F3F4F4F4F5F4FF4
:100080006217730784079507BCF72093DF0030934E
:10009000E0004093E1005093E200089589E288BBBC
:1000A00061E070E080E090E0D9DF88E288BB0895ED
:1000B00020917B0030917C0040917D0050917E002A
:1000C000E2DE20E030E040E050E004C02F5F3F4F30
:1000D0004F4F5F4F6217730784079507BCF7209354
:1000E000E3003093E4004093E5005093E600089568
:1000F0001F9318BA81E087BB19E218BB68EE73E062
:1001000080E090E0ABDF83E087BB18BB61E070E08C
:1001100080E090E0A3DF1F91089583E087BB89E230
:1001200088BB0895662391F4853011F417B83EC05A
:10013000823011F481E039C0843011F482E035C09E
:10014000833099F18A3091F58DE02FC06130A1F4B0
:10015000853011F480E929C0823011F481E925C08D
:10016000843011F482E921C0833011F483E91DC089
:100170008A30E1F48DE919C06230C1F4853011F4A0
:1001800080E813C0823011F481E80FC0843011F48C
:1001900082E80BC0833011F483E807C08A3011F481
:1001A0008DE803C08B3011F48FE887B986EC86B9EF
:1001B0003699FECF84B195B19C0140E050E0209388
:1001C000B3003093B4004093B5005093B60066235B
:1001D00019F58091BB009091BC00A091BD00B09139
:1001E000BE00281B390B4A0B5B0B2093B3003093E6
:1001F000B4004093B5005093B60057FF08C010926A
:10020000B3001092B4001092B5001092B60020E234
:100210003EE440E050E05AC06130A1F58091BF005B
:100220009091C000A091C100B091C200281B390B71
:100230004A0B5B0B2093B3003093B4004093B5009E
:100240005093B60057FF08C01092B3001092B4004C
:100250001092B5001092B6002AE030E040E050E085
:100260006091B3007091B4008091B5009091B60098
:100270000ADE6093B3007093B4008093B50090934E
:10028000B6003AC06230C1F58091C3009091C400BD
:10029000A091C500B091C600281B390B4A0B5B0B1F
:1002A0002093B3003093B4004093B5005093B60050
:1002B00057FF08C01092B3001092B4001092B5001E
:1002C0001092B6002CE434E040E050E06091B300BE
:1002D0007091B4008091B5009091B600D4DD2FEFFD
:1002E00033E040E050E007DE2093B3003093B400E9
:1002F0004093B5005093B6006091B3007091B40084
:100300008091B5009091B60008951092BB001092B4
:10031000BC001092BD001092BE0060E08AE002DFD7
:1003200084B195B1A0E0B0E08093BB009093BC0095
:10033000A093BD00B093BE001092BF001092C00009
:100340001092C1001092C20061E08AE0EBDE84B13D
:1003500095B1A0E0B0E08093BF009093C000A0935F
:10036000C100B093C2001092C3001092C40010925A
:10037000C5001092C60062E08AE0D4DE84B195B177
:10038000A0E0B0E08093C3009093C400A093C500A8
:10039000B093C600089589E288BB61E070E080E018
:1003A00090E05CDE1092A6001092A7001092A800C8
:1003B0001092A90021C08BE288BB64E170E080E06C
:1003C00090E076DE89E288BB69E170E080E090E051
:1003D00045DE8091A6009091A700A091A800B09161
:1003E000A9000196A11DB11D8093A6009093A700BE
:1003F000A093A800B093A9008091A6009091A700B7
:10040000A091A800B091A9000A97A105B1059CF29E
:1004100008951F93182F109220010BC0BCDF6AEFC4
:1004200070E080E090E01ADE809120018F5F809381
:10043000200180912001811788F31F910895E1998F
:10044000FECF1CBA90E09FBB8EBB6DBBE29AE19AD7
:100450000895E199FECF90E09FBB8EBBE09A8DB3EB
:1004600090E00895AF92BF92CF92DF92EF92FF9209
:100470000F931F9361E280E0E2DF81E0EADF8F3FCC
:1004800021F081E0E6DF8093800082E0E2DF8F3FB1
:1004900069F082E0DEDF90E0A0E0B0E080936A00E7
:1004A00090936B00A0936C00B0936D0083E0D1DF5C
:1004B0008F3F09F45FC083E0CCDFA82EBB24CC249F
:1004C000DD24A0926F00B0927000C0927100D092B3
:1004D00072001092E7001092E8001092E90010926A
:1004E000EA00E0906A00F0906B0000916C001091BF
:1004F0006D00EE0CFF1C001F111F84E690E0A0E0D1
:10050000B0E0E80EF91E0A1F1B1FE0929100F09266
:100510009200009393001093940025E730E040E0B0
:1005200050E0C801B701AFDCA6019501ACDC20EEBC
:100530003EE240E050E0DFDC59016A0125E230E0B4
:1005400040E050E0C801B7019EDC64577E40804027
:10055000904028E730E040E050E0CDDCA20EB31E32
:10056000C41ED51EA0927300B0927400C092750094
:10057000D092760080918000833081F480916F006A
:1005800090917000A0917100B091720080937300FF
:1005900090937400A0937500B093760084E059DFC7
:1005A00080936E0085E055DF8F3F91F085E051DF4D
:1005B00090E064E670E055DCAA2797FDA095BA2F7D
:1005C00080938D0090938E00A0938F00B093900045
:1005D00080E13FDF8F3F21F080E13BDF809314011A
:1005E00081E137DF8F3F21F081E133DF8093190113
:1005F00084E22FDF8F3F21F084E22BDF8093210103
:1006000085E227DF8F3F21F085E223DF80932201FF
:1006100086E21FDF8F3F39F086E21BDF90E0909388
:1006200087008093860080E214DF8F3F21F080E214
:1006300010DF8093880081E20CDF8F3F21F081E2A0
:1006400008DF8093600082E204DF8F3F21F082E2C6
:1006500000DF8093610083E2FCDE8F3F91F083E254
:10066000F8DE90E064E670E0FCDBAA2797FDA09539
:10067000BA2F8093890090938A00A0938B00B09347
:100680008C001F910F91FF90EF90DF90CF90BF9063
:10069000AF9008956F927F928F929F92AF92BF9288
:1006A000CF92DF92EF92FF920F931F933B014C0189
:1006B0008091E7009091E800A091E900B091EA00F4
:1006C0000196A11DB11D8093E7009093E800A093CF
:1006D000E900B093EA0083309105A105B105E9F482
:1006E00060926F0070927000809271009092720020
:1006F0002DE730E040E050E0C401B301C4DB24E664
:1007000030E040E050E0F7DB20938200309383003C
:10071000409384005093850036C00497A105B1052D
:1007200094F1E0906F00F0907000009171001091D2
:1007300072002BE030E040E050E0C801B701A3DBDD
:100740002AE030E040E050E0D6DB261537054805CA
:1007500059050CF41BC1C801B701F3E0660F771F00
:10076000881F991FFA95D1F76E0D7F1D801F911F6D
:100770002AE030E040E050E0BEDB621673068406FB
:1007800095063CF503C120916F00309170004091B7
:10079000710050917200CA01B901E2E0660F771F43
:1007A000881F991FEA95D1F7620F731F841F951F49
:1007B000660D771D881D991D26E030E040E050E071
:1007C0009ADB20936F003093700040937100509338
:1007D0007200E0906A00F0906B0000916C00109144
:1007E0006D00EE0CFF1C001F111F84E690E0A0E0DE
:1007F000B0E0E80EF91E0A1F1B1FE0929100F09274
:100800009200009393001093940060906F0070909A
:100810007000809071009090720025E230E040E01E
:1008200050E0C801B7012FDB64577E408040904004
:1008300028E730E040E050E05EDB59016A0125E73F
:1008400030E040E050E0C401B3011DDBA801970196
:100850001ADB20EE3EE240E050E04DDB2A0D3B1D6E
:100860004C1D5D1D20937300309374004093750000
:1008700050937600261537054805590544F46092D3
:10088000730070927400809275009092760097FECB
:100890000CC081E090E0A0E0B0E080936F00909306
:1008A0007000A0937100B093720080916F009091DE
:1008B0007000A0917100B09172008F3F9105A10569
:1008C000B10564F08EEF90E0A0E0B0E080936F009F
:1008D00090937000A0937100B093720020916F000C
:1008E000309170004091710050917200809195009C
:1008F00090919600A0919700B09198002817390721
:100900004A075B0799F0622F83E099DD80916F00C1
:1009100090917000A0917100B09172008093950049
:1009200090939600A0939700B09398008091E70071
:100930009091E800A091E900B091EA000397A10529
:10094000B1056CF480916F0090917000A0917100DE
:10095000B0917200880F991FAA1FBB1F0FC0809112
:100960008000833099F480916F0090917000A09185
:100970007100B09172000297A109B10980937300D0
:1009800090937400A0937500B09376001F910F911F
:10099000FF90EF90DF90CF90BF90AF909F908F909F
:1009A0007F906F900895982F882339F483E08ABD53
:1009B00080E88CBD89E288BB089581E88CBD83E224
:1009C0008ABD81E083BF92BF98BD88E089BF1CBC0F
:1009D000089580E0E8DF08951F93182F80E439DD43
:1009E000809381008F3F19F480E48093810080918F
:1009F00081008F5F80938100803B18F081E48093B9
:100A00008100612F809181001ADD6091810080E476
:100A100016DD1F9108951F9364EF71E080E090E070
:100A20001DDBB9DC1092F0001092F1001092F20080
:100A30001092F3001092B7001092B8001092B90013
:100A40001092BA0069C060E084E06CDB645F7140C2
:100A50008040904014F41092D30060E084E062DBA8
:100A600069557B41804090400CF443C08091D30095
:100A7000882309F03EC08091F0009091F100A09190
:100A8000F200B091F30086309105A105B10524F084
:100A90000997A105B10509F47EDC8091F0009091E1
:100AA000F100A091F200B091F3000196A11DB11DDB
:100AB0008093F0009093F100A093F200B093F300C4
:100AC0008093800087309105A105B1053CF00A971D
:100AD000A105B10519F086E0809380001092B7005F
:100AE0001092B8001092B9001092BA0081E0809381
:100AF000D3008091B7009091B800A091B900B09157
:100B0000BA000196A11DB11D8093B7009093B80063
:100B1000A093B900B093BA008091B7009091B8004B
:100B2000A091B900B091BA0088559240A040B04061
:100B30000CF489CF81E06DDC2EDC1092B7001092AE
:100B4000B8001092B9001092BA0059C060E084E079
:100B5000E9DA645F71408040904014F41092D30051
:100B600060E084E0DFDA69557B4180409040A4F189
:100B70008091D300882381F580916A0090916B0069
:100B8000A0916C00B0916D00181619061A061B068C
:100B90001CF54597A105B105A4F0FDDB80916A0025
:100BA00090916B00A0916C00B0916D000297A1092B
:100BB000B10980936A0090936B00A0936C00B0938E
:100BC0006D001092B7001092B8001092B900109208
:100BD000BA0081E08093D3008091B7009091B80073
:100BE000A091B900B091BA000196A11DB11D8093EA
:100BF000B7009093B800A093B900B093BA00809169
:100C0000B7009091B800A091B900B091BA00885592
:100C10009240A040B0400CF499CF82E0FADBBBDBFD
:100C20001092B7001092B8001092B9001092BA005A
:100C300055C060E084E076DA645F714080409040A7
:100C400014F41092D30060E084E06CDA69557B41C3
:100C50008040904084F18091D300882361F5809199
:100C60006A0090916B00A0916C00B0916D008A3F7A
:100C70009105A105B105FCF48EDB80916A0090918D
:100C80006B00A0916C00B0916D000196A11DB11D8B
:100C900080936A0090936B00A0936C00B0936D00FA
:100CA0001092B7001092B8001092B9001092BA00DA
:100CB00081E08093D3008091B7009091B800A0911B
:100CC000B900B091BA000196A11DB11D8093B70083
:100CD0009093B800A093B900B093BA008091B70088
:100CE0009091B800A091B900B091BA008855924097
:100CF000A040B0400CF49DCF83E08BDB4CDB109226
:100D0000B7001092B8001092B9001092BA004EC00D
:100D100060E084E007DA645F71408040904014F442
:100D20001092D30060E084E0FDD969557B4180409A
:100D300090404CF18091D300882329F580916E007A
:100D4000882309F1853360F026DB80916E0090E006
:100D500069E070E086D86AE070E0BAD860936E000F
:100D60001092B7001092B8001092B9001092BA0019
:100D70001092E7001092E8001092E9001092EA0049
:100D800081E08093D3008091B7009091B800A0914A
:100D9000B900B091BA000196A11DB11D8093B700B2
:100DA0009093B800A093B900B093BA008091B700B7
:100DB0009091B800A091B900B091BA0088559240C6
:100DC000A040B0400CF4A4CF84E023DBE4DA10921E
:100DD000B7001092B8001092B9001092BA0052C039
:100DE00060E084E09FD9645F71408040904014F4DB
:100DF0001092D30060E084E095D969557B41804032
:100E000090406CF18091D300882349F580916E0069
:100E10008F3F29F1883E68F4BEDA80916E0090E041
:100E20006BE070E01ED86AE070E052D860936E000C
:100E300003C08EEF80936E001092B7001092B8003E
:100E40001092B9001092BA001092E7001092E800D8
:100E50001092E9001092EA0081E08093D300809123
:100E6000B7009091B800A091B900B091BA00019676
:100E7000A11DB11D8093B7009093B800A093B90055
:100E8000B093BA008091B7009091B800A091B900DA
:100E9000B091BA0088559240A040B0400CF4A0CF69
:100EA00085E0B7DA78DA109221011092B70010923B
:100EB000B8001092B9001092BA003EC060E084E021
:100EC00031D9645F71408040904014F41092D30097
:100ED00060E084E027D969557B4180409040CCF0A8
:100EE0008091D3008823A9F480912101823030F4CD
:100EF00052DA809121018F5F809321011092B70017
:100F00001092B8001092B9001092BA0081E080935C
:100F1000D3008091B7009091B800A091B900B09132
:100F2000BA000196A11DB11D8093B7009093B8003F
:100F3000A093B900B093BA008091B7009091B80027
:100F4000A091B900B091BA0088559240A040B0403D
:100F50000CF4B4CF86E05DDA1EDA109287001092AE
:100F600086001092B7001092B8001092B90010924B
:100F7000BA0044C060E084E0D5D8645F714080402E
:100F8000904014F41092D30060E084E0CBD869550F
:100F90007B4180409040FCF08091D3008823D9F4BD
:100FA0008091860090918700029750F4F4D9809147
:100FB0008600909187000196909387008093860029
:100FC0001092B7001092B8001092B9001092BA00B7
:100FD00081E08093D3008091B7009091B800A091F8
:100FE000B900B091BA000196A11DB11D8093B70060
:100FF0009093B800A093B900B093BA008091B70065
:101000009091B800A091B900B091BA008855924073
:10101000A040B0400CF4AECF8091F0009091F10070
:10102000A091F200B091F3000097A105B105A9F1DC
:10103000809180008A3031F462E080E200DA83E05F
:101040008093800080918000843049F460E081E2E8
:10105000F6D91092600082E0809380000AC081E29D
:10106000F8D98F3F31F06FEF81E2E9D981E08093C9
:10107000600080918000853039F464E685E2DFD934
:1010800083E08093800009C085E2E3D98F3F29F097
:101090006FEF85E2D4D9109222016091800081E047
:1010A000CED980916A0090916B00A0916C00B091B4
:1010B0006D004497A105B10564F484E190E0A0E0DF
:1010C000B0E080936A0090936B00A0936C00B093A3
:1010D0006D0080916A0090916B00A0916C00B091BE
:1010E0006D008B3F9105A105B10564F08AEF90E09A
:1010F000A0E0B0E080936A0090936B00A0936C0036
:10110000B0936D0060916A0082E099D980916E0081
:10111000843318F484E380936E0080916E008F3FD7
:1011200019F48EEF80936E0060916E0084E087D991
:1011300060E082E0F7D760938D0070938E0080931B
:101140008F009093900024E630E040E050E0D3D64A
:101150002093F400622F85E072D9109121011130A3
:1011600029F461E084E26BD910932101809121017F
:10117000823029F460E084E262D9109221018091EA
:10118000860090918700019739F460E086E257D994
:1011900010928700109286008091860090918700BF
:1011A000029749F461E086E24AD981E090E09093A9
:1011B00087008093860087E02CD9EDD81092EC0050
:1011C0001092ED001092EE001092EF001092B70016
:1011D0001092B8001092B9001092BA005FC08091CE
:1011E000EC009091ED00A091EE00B091EF0001961F
:1011F000A11DB11D8093EC009093ED00A093EE0033
:10120000B093EF008D5D9540A040B0405CF186E06A
:10121000E3DB6FEF80E013D96FEF81E010D96FEF60
:1012200082E00DD96FEF83E00AD96FEF84E007D930
:101230006FEF85E004D96FEF84E201D96FEF81E2AF
:10124000FED86FEF85E2FBD86FEF86E2F8D8A3D81F
:10125000A2D8A1D8A0D89FD89ED89DD89CD89BD8DA
:101260009AD8FFCF60E084E05DD769557B4180402C
:1012700090400CF0B4CF8091B7009091B800A0914D
:10128000B900B091BA000196A11DB11D8093B700BD
:101290009093B800A093B900B093BA008091B700C2
:1012A0009091B800A091B900B091BA0088559240D1
:1012B000A040B040BCF21F9108952F923F924F92F0
:1012C0005F926F927F928F929F92AF92BF92CF92D6
:1012D000DF92EF92FF920F931F9319E218BB61E028
:1012E00070E080E090E0BAD68BE288BB61E070E00D
:1012F00080E090E0B3D661E082E014D728EE33E0DE
:1013000040E050E0C0D520E035E040E050E0F3D5CB
:1013100020939E0030939F004093A0005093A10023
:1013200018BB255F3140404050403CF018BB82E084
:1013300053DB81E18093990073C081E034DB8091BD
:10134000610010916E00813009F049C0812F8695AF
:10135000282E3324442455242091FB003091FC0096
:101360004091FD005091FE00612E7724882499243D
:10137000EE24FF248701AA24BB24650115C0C60101
:10138000B501661977098809990924E630E040E03B
:1013900050E0B1D5220D331D441D551D28BD0894C4
:1013A000E11CF11C011D111DA60CB71CC81CD91C89
:1013B00083E3E816F104010511050CF32093FB000B
:1013C0003093FC004093FD005093FE00E092F70044
:1013D000F092F8000093F9001093FA0021C0612FF9
:1013E00070E080E090E02091F7003091F8004091AB
:1013F000F9005091FA0047D524E630E040E050E093
:101400007AD5812F8695280F311D411D511D2093BE
:10141000FB003093FC004093FD005093FE0018BD8C
:101420001F910F91FF90EF90DF90CF90BF90AF9002
:101430009F908F907F906F905F904F903F902F90F4
:10144000089589E288BB61E070E080E090E006D614
:1014500060E083E067D624E030E040E050E04BD528
:10146000209306013093070140930801509309012E
:1014700060E085E057D624E030E040E050E03BD526
:1014800020930A0130930B0140930C0150930D01FE
:101490008091060190910701A0910801B091090186
:1014A0008C3261E0960760E0A60760E0B60774F44E
:1014B0002C3261E0360760E0460760E0560734F4FE
:1014C00081E080930E0181E090E00895255F314036
:1014D000404050401CF083E090E00895855F9140CB
:1014E000A040B0401CF082E090E0089581E090E0E0
:1014F0000895EF92FF920F931F9360ED77E080E0E5
:1015000090E0ACD581E08093990080937F00FDD678
:1015100060E084E007D6655F7140804090401CF039
:1015200084E0809399009ED780E293D7823009F0BF
:101530005CC08FD78F3F09F445C080916A009091BD
:101540006B00A0916C00B0916D00E0906F00F09086
:101550007000009171001091720080359105A10515
:10156000B10594F08F54809323016AE0A5D4E80E6E
:10157000F11C011D111DE0926F00F09270000093AC
:101580007100109372001EC083518093230122E4E6
:1015900030E0281B3109442737FD4095542FE21ACB
:1015A000F30A040B150BC801B70125E030E040E059
:1015B00050E0A1D420936F003093700040937100ED
:1015C0005093720080916F0090917000A091710013
:1015D000B09172000297A109B109809373009093B2
:1015E0007400A0937500B093760082D513E017BB0A
:1015F00089E288BB60E082E095D59B01AC016093F5
:10160000A2007093A3008093A4009093A5002835B6
:101610008BE1380780E0480780E058071CF482E03F
:101620008093990021583E434040504024F081E08F
:10163000D3D91093990080918D0090918E00A09144
:101640008F00B09190000097A105B10559F460E0BA
:1016500082E068D560938D0070938E0080938F0038
:10166000909390008091890090918A00A0918B00C6
:10167000B0918C000097A105B10541F080938D00D9
:1016800090938E00A0938F00B0939000E0908D0017
:10169000F0908E0000918F001091900020E530E0D6
:1016A00040E050E0C801B701EED324E630E040E06E
:1016B00050E021D420936600309367004093680087
:1016C0005093690025E530E040E050E0C801B701E3
:1016D000DAD324E630E040E050E00DD420936200FD
:1016E000309363004093640050936500AADE8093BA
:1016F00005011092DB001092DC001092DD001092C8
:10170000DE0019C064EF71E080E090E0A7D443D61A
:101710008091DB009091DC00A091DD00B091DE00B3
:101720000196A11DB11D8093DB009093DC00A09376
:10173000DD00B093DE0060919900262F30E040E09C
:1017400050E08091DB009091DC00A091DD00B09131
:10175000DE0082179307A407B507A4F26230F0F702
:101760001092B7001092B8001092B9001092BA000F
:101770001EC060E084E0D6D469557B418040904033
:101780001CF085E029D947D98091B7009091B80025
:10179000A091B900B091BA000196A11DB11D80932E
:1017A000B7009093B800A093B900B093BA008091AD
:1017B000B7009091B800A091B900B091BA00815AD9
:1017C0009440A040B040ACF280918800882319F08A
:1017D00083E080938000DFD5DED5DDD5DCD5809138
:1017E0000E01882321F0D7D5D6D5D5D5D4D5809173
:1017F000D4009091D500A091D600B091D700019669
:10180000A11DB11D8093D4009093D500A093D60064
:10181000B093D7008091100190911101A091120115
:10182000B09113010196A11DB11D809310019093F9
:101830001101A0931201B0931301CBD860E084E0B2
:1018400071D49B01AC0160939A0070939B008093CC
:101850009C0090939D008091660090916700A091FC
:101860006800B0916900281739074A075B07A4F49C
:1018700029553B41404050407CF08091F6008F5FFD
:101880008093F600863040F086D568EE73E080E005
:1018900090E0E4D31092F60020919A0030919B00E2
:1018A00040919C0050919D0080916600909167004E
:1018B000A0916800B0916900281739074A075B07B3
:1018C000ECF18091D3008823C9F580910E01882323
:1018D000A9F48091620090916300A0916400B0919E
:1018E0006500281739074A075B076CF48091F500FB
:1018F0008F5F8093F5008330E8F4B6C0A2DD80935B
:101900000501813019F41092F500AEC09091F500F8
:101910009F5F9093F500833039F4933008F4A4C0AE
:1019200080E1809399009BC1823009F09DC0933083
:1019300008F49AC080E18093990096C0245F3140FA
:10194000404050406CF41092D30081E080937F00BF
:101950001092D4001092D5001092D6001092D700A9
:101960008091D4009091D500A091D600B091D7007D
:10197000833A9105A105B10584F08091D3008130AF
:1019800061F480918000833041F08091600081306B
:1019900021F482E080937F0067C080910F0188234B
:1019A00009F025CF8091C7009091C800A091C9008F
:1019B000B091CA008D529140A040B04008F417CFBA
:1019C0008091100190911101A0911201B091130129
:1019D000895E9340A040B0400CF409CF809189000B
:1019E00090918A00A0918B00B0918C000097A10586
:1019F000B10509F4FCCE60E082E094D37B018C0158
:101A000060938D0070938E0080938F009093900070
:101A100020E530E040E050E036D224E630E040E01F
:101A200050E069D2209366003093670040936800CD
:101A30005093690025E530E040E050E0C801B7016F
:101A400022D224E630E040E050E055D220936200FC
:101A500030936300409364005093650084E0BCD7EA
:101A600081E080930F01C3CE80911A01813009F487
:101A7000F6C023DC61E070E080E090E0EFD21092ED
:101A8000CB001092CC001092CD001092CE0010929C
:101A9000CF001092D0001092D1001092D20080910D
:101AA000C7009091C800A091C900B091CA000196EA
:101AB000A11DB11D8093C7009093C800A093C900D9
:101AC000B093CA008091CB009091CC00A091CD0042
:101AD000B091CE000196A11DB11D8093CB009093D3
:101AE000CC00A093CD00B093CE0061E084E01AD387
:101AF00060939A0070939B0080939C0090939D004C
:101B0000685B7B40804090400CF083C080918600F1
:101B100090918700892B79F5209182003091830084
:101B20004091840050918500E0907300F090740023
:101B300000917500109176002E153F054007510762
:101B4000D0F48091CB009091CC00A091CD00B091C9
:101B5000CE00281739074A075B0768F48E159F05E2
:101B6000A007B10744F480918000823009F4AACF25
:101B7000843009F4A7CF80918000863009F03FC0FF
:101B80008091C7009091C800A091C900B091CA008F
:101B90002091CB003091CC004091CD005091CE00EF
:101BA0000697A105B10518F4CA01B90126C08091B4
:101BB000730090917400A0917500B0917600E09050
:101BC000CF00F090D0000091D1001091D200821788
:101BD0009307A407B5077CF0E114F1040105110592
:101BE00009F070CF2093CF003093D0004093D10004
:101BF0005093D20067CFC801B7014CD530C08130B7
:101C000021F080917F00823051F581E080937F0048
:101C100026C090918000963009F454CF80917F00C7
:101C2000823009F44FCF913009F44CCF2091CB0092
:101C30003091CC004091CD005091CE008091730046
:101C400090917400A0917500B0917600821793076F
:101C5000A407B5070CF036CF81E08093D300B9D646
:101C60001DD26BE470E080E090E0F8D189E288BB9F
:101C700020912201222309F450C08091C700909145
:101C8000C800A091C900B091CA000597A105B1058F
:101C900008F443C0822F90E06AE070E0E2D0AA2707
:101CA00097FDA095BA2FBC01CD01D8D1809121011B
:101CB000813099F585E090E0A0E0B0E019C08BE2BA
:101CC00088BB64E170E080E090E0F2D189E288BBFB
:101CD00069E170E080E090E0C1D18091A600909130
:101CE000A700A091A800B091A9000197A109B1098E
:101CF0008093A6009093A700A093A800B093A9009A
:101D00008091A6009091A700A091A800B091A90091
:101D1000181619061A061B0694F28091D300882320
:101D200069F480918000863049F06091CB00709119
:101D3000CC008091CD009091CE00ACD462E08BE0DD
:101D4000F1D124E630E040E050E09DD06856744781
:101D5000804090402DE630E040E050E0CCD0209331
:101D600015013093160140931701509318012C333D
:101D70003105410551052CF083E02ED681E080939A
:101D80001A012091150130911601409117015091CF
:101D90001801283331054105510514F410921A0138
:101DA00080911A01813019F482E180939900109298
:101DB000D4001092D5001092D6001092D700109245
:101DC00010011092110110921201109213018091D2
:101DD000140190E0A0E0B0E082179307A407B507D4
:101DE0002CF420931401622F80E129D360919E008E
:101DF00070919F008091A0009091A1002AE030E0B6
:101E000040E050E078D08091190190E0A0E0B0E08F
:101E100082179307A407B5072CF420931901622FAA
:101E200081E10DD380919900882309F4E0CC64E628
:101E300070E080E090E012D180919900803111F43F
:101E400081E0E7D280919900813111F482E0E1D202
:101E500080919900823111F483E0DBD210929900D5
:101E6000C6CC5527002480FF02C0060E571F660F00
:101E7000771F6115710521F096958795009799F761
:101E8000952F802D0895FF27EE27BB27AA2760FFF7
:101E900004C0A20FB31FE41FF51F220F331F441FFE
:101EA000551F969587957795679589F700977607DB
:101EB00071F7CF01BD010895991B79E004C0991F06
:101EC000961708F0961B881F7A95C9F78095089594
:101ED00097FB092E07260AD077FD04D027D006D01D
:101EE00000201AF4709561957F4F0895F6F790954C
:101EF00081959F4F089597FB092E05260ED057FD1B
:101F000004D028D00AD0001C38F450954095309564
:101F100021953F4F4F4F5F4F0895F6F7909580956D
:101F2000709561957F4F8F4F9F4F0895AA1BBB1BE4
:101F300051E107C0AA1FBB1FA617B70710F0A61BC9
:101F4000B70B881F991F5A95A9F780959095BC01EA
:101F5000CD010895A1E21A2EAA1BBB1BFD010DC0E5
:101F6000AA1FBB1FEE1FFF1FA217B307E407F50749
:101F700020F0A21BB30BE40BF50B661F771F881F25
:101F8000991F1A9469F760957095809590959B01BB
:0A1F9000AC01BD01CF010895FFCFA1
:101F9A0001017C1500007017000050000000FE4689
:101FAA00000000CD000000640000000100000001F4
:081FBA0002FF580000000100C5
:00000001FF
